:100000009428003803198F28A8002008840021189C
:100010008317A001A101A81B15280008A000A81C97
:100020008F28840A0008A1008F281A200005031DCC
:10003000A00A8F2800308A00280807398207013477
:10004000023404340834103420344034803421081D
:1000500020040319A00A8030201AA1062019A10645
:10006000A018A106210DA00DA10D8F28A301A200AB
:10007000FF30A207031CA307031C8F280330A10035
:10008000DF3044203828A101E83EA000A109FC305F
:10009000031C4D28A00703184A28A0076400A10FDD
:1000A0004A2820185328A01C572800005728080069
:1000B000A20001306328A20006306328A2000430A9
:1000C0006328A2000530A80023082102031D6A2826
:1000D00022082002043003180130031902302805D9
:1000E000031DFF308F28A501A4011030A600210DAB
:1000F000A40DA50D2208A4022308031C230FA502AA
:10010000031889282208A40723080318230FA5072A
:100110000310A00DA10DA60B772820088F288313AC
:10012000031383126400080083168701850183127C
:10013000BA01BB013A08A0003B08A100A3013C3072
:100140008A0158208A11031D2C2E3B088A11031D99
:10015000B5293A08A2003B3C8A11031CB5290310BB
:10016000220DA2078A11C420A000A20A8A11C4206D
:10017000A100A20A8A11C4208A0101202008D4000B
:100180002108D5008A11B52901308A0022080029EA
:1002000082070134003400340234003400340334F3
:100210000034003404340034003405340034003435
:100220000634003400340734003400340834003419
:1002300000340934003400340A34003400340B3400
:10024000003400340C3400340034043400340034FE
:1002500003340034003405340034003407340034EF
:1002600000340234003400340934003400340634DD
:10027000003400340B34003400340A3400340034C9
:100280000134003400340C340034003408340034B9
:1002900000340234003400340534003400340734B0
:1002A000003400340A3400340034043400340034A0
:1002B0000634003400340B34003400340834003485
:1002C0000034093400340034033400340034013481
:1002D000003400340C34003400340A340034003468
:1002E0000234003400340434003400340C3400345C
:1002F0000034053400340034083400340034013450
:100300000034003403340034003406340034003444
:100310000B34003400340934003400340734003422
:10032000003402340034003406340034003407341E
:10033000003400340334003400340C34003400340E
:1003400001340034003404340034003409340034FF
:1003500000340534003400340834003400340B34E5
:10036000003400340A34003400345408A000550826
:10037000A100A30101308A0161208A11031D3D2AD9
:100380008316C80A0319C90A48088312A0008316F5
:1003900049088312A100A30105308A015B208A115C
:1003A000031DD6298316C801C90183128316490883
:1003B0008A118312031DF52983164808053C8A110A
:1003C0008312031CF5298A11E921E200E3018A1155
:1003D000F52901308A0083164808831282073234D7
:1003E0003C3446341E345034283483165C0883125F
:1003F000A00083165D088312A1008A01272020082F
:100400008316DC00831221088316DD005C0883124A
:10041000A00083165D088312A1001130A200A30181
:100420008A01732024088316DE00831225088316B0
:10043000DF0001305E07E0005F080318013EE100C5
:100440008312D601D7015608A0005708A1008316D1
:1004500061088312A3008316600883128A01582062
:100460008A11031D3B2A8A112E26D60A0319D70AA0
:100470008A11031D232A8A11262E5408A00055082C
:10048000A100A30102308A0161208A11031DC52A3F
:100490008316D60A0319D70A56088312A0008316BA
:1004A00057088312A100A30105308A015B208A113D
:1004B000031D5E2A8316D601D701831283165708BF
:1004C0008A118312031D7D2A83165608053C8A1162
:1004D0008312031C7D2A8A117122F800F9018A1106
:1004E0007D2A02308A0083165608831282077D34E3
:1004F0004B34D23432342C34AF3483166208831236
:10050000A000831663088312A1008A012720200817
:100510008316E200831221088316E3006208831227
:10052000A000831663088312A1001330A200A30168
:100530008A01732024088316E40083122508831699
:10054000E50001306407CA0065080318013ECB00CE
:100550008312DA01DB015A08A0005B08A1008316B0
:100560004B088312A30083164A0883128A0158207D
:100570008A11031DC32A8A117626DA0A0319DB0AB7
:100580008A11031DAB2A8A11262E5408A000550893
:10059000A100A30103308A0161208A11031D252BCC
:1005A0009030FE000130FF007E08A0007F08A1000F
:1005B000A30196308A015E208A11031DEF2A8A1159
:1005C0008F263230FE0200308A110318EB2A013EDA
:1005D0008A110318EF2AFF028A110318D42A5A300D
:1005E000FE00FF017E08A0007F08A100A3013230B9
:1005F0008A015E208A11031D0D2B8A118F2605307A
:10060000FE0200308A110318092B013E8A110318DB
:100610000D2BFF028A110318F22A0130D800D901EC
:100620005808A0005908A100A30107308A015820EA
:100630008A11031D232B8A118F26D80A0319D90A80
:100640008A11031D102B8A11262E5408A00055086C
:10065000A100A30104308A0161208A11031DAF2B80
:100660008316D80A0319D90A58088312A0008316E2
:1006700059088312A100A30105308A015B208A1169
:10068000031D462B8316D801D901831283165908FE
:100690008A118312031D672B83165808053C8A11A3
:1006A0008312031C672B8A115B238316A000A10110
:1006B00083128A11672B03308A008316580883122D
:1006C0008207323496343C345A342C344634831600
:1006D0005A088312A00083165B088312A1008A01C6
:1006E000272020088316DA00831221088316DB00F6
:1006F0005A088312A00083165B088312A1001930E8
:10070000A200A3018A01732024088316DC0083124F
:1007100025088316DD0001305C07DE005D08031844
:10072000013EDF008312DA01DB015A08A0005B08FA
:10073000A10083165F088312A30083165E0883124C
:100740008A0158208A11031DAD2B8A11B026DA0ABE
:100750000319DB0A8A11031D952B8A11262E5408D2
:10076000A0005508A100A30105308A0161208A116B
:10077000031D392C8316B80A0319B90A38088312E5
:10078000A000831639088312A100A30105308A0155
:100790005B208A11031DD02B8316B801B901831287
:1007A000831639088A118312031DF12B831638082A
:1007B000053C8A118312031CF12B8A11E523831651
:1007C000A600A70183128A11F12B03308A00831639
:1007D0003808831282077D344B346E343234AF34A0
:1007E000963483163A088312A00083163B088312BE
:1007F000A1008A01272020088316BA00831221084D
:100800008316BB003A088312A00083163B088312AC
:10081000A1000A30A200A3018A01732024088316D4
:10082000BC00831225088316BD0001303C07BE00C2
:100830003D080318013EBF008312CA01CB014A08DC
:10084000A0004B08A10083163F088312A300831663
:100850003E0883128A0158208A11031D372C8A1101
:10086000E227CA0A0319CB0A8A11031D1F2C8A1119
:10087000262E5408A0005508A100A30106308A01C5
:1008800061208A11031D982CC830E800E90168082E
:10089000A0006908A100A30164308A015E208A11CA
:1008A000031D622C8A1502251930E80200308A11D6
:1008B00003185E2C013E8A110318622CE9028A118A
:1008C0000318472C6430E800E9016808A0006908B3
:1008D000A100A3013C308A015E208A11031D802CF7
:1008E0008A1502250A30E80200308A1103187C2C90
:1008F000013E8A110318802CE9028A110318652C25
:100900000130CC00CD014C08A0004D08A100A3018E
:1009100007308A0158208A11031D962C8A1502255A
:10092000CC0A0319CD0A8A11031D832C8A11262EA5
:100930005408A0005508A100A30107308A016120D6
:100940008A11031DE12C6430EC00ED016C08A0005D
:100950006D08A100A30146308A015E208A11031DA3
:10096000C12C8A1561260530EC0200308A1103186B
:10097000BD2C013E8A110318C12CED028A11031807
:10098000A62C4630E400E5016408A0006508A1003B
:10099000A30128308A015E208A11031DDF2C8A15ED
:1009A00044240530E40200308A110318DB2C013E98
:1009B0008A110318DF2CE5028A110318C42C8A114E
:1009C000262E5408A0005508A100A30108308A0172
:1009D00061208A11031D3A2D8316C830A200A3019D
:1009E0008312831622088312A00083162308831221
:1009F000A100A30164308A015E208A11031D122D1B
:100A00008A11C92619308316A20200308A11831276
:100A100003180E2D013E8A110318122DA3028A110C
:100A20000318F12C83166430A200A30183128316ED
:100A300022088312A000831623088312A100A301B9
:100A40003C308A015E208A11031D382D8A11C92687
:100A50000A308316A20200308A1183120318342D43
:100A6000013E8A110318382DA3028A110318172D8D
:100A70008A11262E5408A0005508A100A3010930B0
:100A80008A0161208A11031D832D7830EA00EB0171
:100A90006A08A0006B08A100A30164308A015E20EF
:100AA0008A11031D632D8A1567250A30EA0200307A
:100AB0008A1103185F2D013E8A110318632DEB0282
:100AC0008A110318482D6430EA00EB016A08A0007F
:100AD0006B08A100A30132308A015E208A11031D38
:100AE000812D8A1567250A30EA0200308A11031821
:100AF0007D2D013E8A110318812DEB028A11031806
:100B0000662D8A11262E5408A0005508A100A301C5
:100B10000A308A0161208A11031DA62D0130C2000E
:100B2000C3014208A0004308A100A30107308A01C5
:100B300058208A11031DA42D8A158B24C20A03197B
:100B4000C30A8A11031D912D8A11262E5408A00074
:100B50005508A100A3010B308A0161208A11031DF1
:100B6000C92D0130C400C5014408A0004508A100FA
:100B7000A30102308A0158208A11031DC72D8A154E
:100B80009521C40A0319C50A8A11031DB42D8A11BF
:100B9000262E5408A0005508A100A3010C308A019C
:100BA00061208A11031D262E9630EE00EF016E089B
:100BB000A0006F08A100A30164308A015E208A11A1
:100BC000031DF22D8A15A8260A30EE0200308A1184
:100BD0000318EE2D013E8A110318F22DEF028A113F
:100BE0000318D72D6430EE00EF016E08A0006F08E7
:100BF000A100A30132308A015E208A11031D102E4C
:100C00008A15A8260A30EE0200308A1103180C2E2D
:100C1000013E8A110318102EEF028A110318F52DD8
:100C20000130C800C9014808A0004908A100A3017B
:100C300007308A0158208A11031D262E8A15A826FE
:100C4000C80A0319C90A8A11031D132EBA0A031907
:100C5000BB0A8A11031D9A288A01982885018701F9
:100C60006308A30062088A01372004308700630804
:100C7000A30062088A013720023087006308A300BE
:100C800062088A013720013087006308A3006208E8
:100C90008A013720203087006308A30062088A0198
:100CA0003720103087006308A30062088A013720CC
:100CB000083087006308A30062088A0137200430E7
:100CC000850087016308A30062088A01372002308B
:100CD00085006308A30062088A013720013085007F
:100CE0006308A30062088A01372008008501870194
:100CF000073087007908A30078088A013720383048
:100D000087007908A30078088A0137208701073017
:100D100085007908A30078088A013720080085013A
:100D200087017F08A3007E088A01372010308700E2
:100D30007F08A3007E088A01372015308700053020
:100D400085007F08A3007E088A0137203A3087009B
:100D5000023085007F08A3007E088A013720080042
:100D600087018501831621088312A30083162008BA
:100D700083128A0137203F308700073085008316B1
:100D800021088312A3008316200883128A013720CA
:100D9000080087018501831623088312A3008316A8
:100DA000220883128A013720043087008316230823
:100DB0008312A3008316220883128A01372024306D
:100DC0008700831623088312A30083162208831248
:100DD0008A013720043087000430850083162308F9
:100DE0008312A3008316220883128A01372004305D
:100DF000870006308500831623088312A30083161C
:100E0000220883128A0137201430870004308500BD
:100E1000831623088312A3008316220883128A01F3
:100E2000372006308700043085008316230883129C
:100E3000A3008316220883128A0137200530870019
:100E400004308500831623088312A300831622082A
:100E500083128A0137200D30870004308500831605
:100E600023088312A3008316220883128A013720E5
:100E70000530870005308500831623088312A30000
:100E80008316220883128A01372005308700073035
:100E90008500831623088312A30083162208831279
:100EA0008A01372005308700033085008316230828
:100EB0008312A3008316220883128A01372025306B
:100EC000870003308500831623088312A30083164E
:100ED000220883128A0137202130870003308500E1
:100EE000831623088312A3008316220883128A0123
:100EF00037202330870003308500831623088312B0
:100F0000A3008316220883128A013720223087002B
:100F100003308500831623088312A300831622085A
:100F200083128A0137202A30870003308500831618
:100F300023088312A3008316220883128A01372014
:100F40002A30870002308500831623088312A3000D
:100F50008316220883128A0137202A308700023044
:100F60008500831623088312A300831622088312A8
:100F70008A01372005308700053085008316230855
:100F80008312A3008316220883128A0137202A3095
:100F9000870002308500831623088312A30083167E
:100FA000220883128A01372005308700053085002A
:100FB000831623088312A3008316220883128A0152
:100FC0003720080085010430870083162708831224
:100FD000A3008316260883128A0137202030870059
:100FE000831627088312A3008316260883128A011A
:100FF0003720870104308500831627088312A30059
:101000008316260883128A013720023087000430B5
:101010008500831627088312A300831626088312EF
:101020008A01372010308700043085008316270896
:101030008312A3008316260883128A0137208701B2
:1010400006308500831627088312A300831626081E
:1010500083128A013720013087000630850083160D
:1010600027088312A3008316260883128A013720DB
:101070000830870006308500831627088312A300F6
:101080008316260883128A013720870107308500DE
:10109000831627088312A3008316260883128A0169
:1010A0003720043087000730850083162708831215
:1010B000A3008316260883128A0137202030870078
:1010C00007308500831627088312A300831626089D
:1010D00083128A013720223087000730850083166B
:1010E00027088312A3008316260883128A0137205B
:1010F0003030870007308500831627088312A3004D
:101100008316260883128A01372031308700073082
:101110008500831627088312A300831626088312EE
:101120008A0137203830870007308500831627086A
:101130008312A3008316260883128A0137203C30CD
:10114000870007308500831627088312A3008316C3
:10115000260883128A0137203E3087000730850039
:10116000831627088312A3008316260883128A0198
:1011700037203F3087000730850083162708831209
:10118000A3008316260883128A0137203B3087008C
:1011900007308500831627088312A30083162608CC
:1011A00083128A0137201F3087000730850083169D
:1011B00027088312A3008316260883128A0137208A
:1011C0003F30870003308500831627088312A30071
:1011D0008316260883128A0137203D3087000330AA
:1011E0008500831627088312A3008316260883121E
:1011F0008A0137202F3087000330850083162708A7
:101200008312A3008316260883128A0137203F30F9
:10121000870001308500831627088312A3008316F8
:10122000260883128A0137203E308700013085006E
:10123000831627088312A3008316260883128A01C7
:101240003720373087000130850083162708831246
:10125000A3008316260883128A0137203F308700B7
:101260008501831627088312A3008316260883129C
:101270008A0137203B3087008501831627088312B7
:10128000A3008316260883128A0137201F308700A7
:10129000831627088312A3008316260883128A0167
:1012A00037201D308700831627088312A30083167A
:1012B000260883128A0137200F30870083162708FB
:1012C0008312A3008316260883128A0137200E306A
:1012D0008700831627088312A3008316260883122B
:1012E0008A01372007308700831627088312A3005E
:1012F0008316260883128A0137200330870083165D
:1013000027088312A3008316260883128A01372038
:1013100001308700831627088312A300831626084E
:1013200083128A0137208701080083169630A800AF
:10133000A9018312850104308700831629088312CE
:10134000A3008316280883128A01372006308700FD
:10135000831629088312A3008316280883128A01A2
:10136000372005308700831629088312A3008316CF
:10137000280883128A013720253087008316290820
:101380008312A3008316280883128A013720353080
:101390008700831629088312A30083162808831266
:1013A0008A0137203D308700831629088312A30065
:1013B0008316280883128A013720353087000430CD
:1013C0008500831629088312A30083162808831238
:1013D0008A013720353087000630850083162908BA
:1013E0008312A3008316280883128A013720353020
:1013F000870005308500831629088312A300831611
:10140000280883128A01372087018501831629085D
:101410008312A3008316280883128A0137203530EF
:10142000870005308500831629088312A3008316E0
:10143000280883128A01372087018501831629082D
:101440008312A3008316280883128A0137203530BF
:10145000870005308500831629088312A3008316B0
:10146000280883128A0137208701850183162908FD
:101470008312A3008316280883128A0137200130C3
:101480008500831629088312A30083162808831277
:101490008A01372002308500831629088312A300B1
:1014A0008316280883128A013720063085008316A8
:1014B00029088312A3008316280883128A01372083
:1014C0000230850020308700831629088312A3008C
:1014D0008316280883128A013720023085001030D5
:1014E0008700831629088312A30083162808831215
:1014F0008A013720023085001830870083162908BA
:101500008312A3008316280883128A013720023031
:10151000850011308700831629088312A3008316E3
:10152000280883128A013720023085001330870093
:10153000831629088312A3008316280883128A01C0
:101540003720153087000230850083162908831262
:10155000A3008316280883128A013720870185019A
:10156000831629088312A3008316280883128A0190
:101570003720153087000230850083162908831232
:10158000A3008316280883128A013720870185016A
:10159000831629088312A3008316280883128A0160
:1015A0003720153087000230850083162908831202
:1015B000A3008316280883128A013720870185013A
:1015C000831629088312A3008316280883128A0130
:1015D000372004308700831629088312A30083165E
:1015E000280883128A0137202430870083162908AF
:1015F0008312A3008316280883128A01372024301F
:10160000870004308500831629088312A3008316FF
:10161000280883128A01372026308700043085008D
:10162000831629088312A3008316280883128A01CF
:101630003720343087000430850083162908831250
:10164000A3008316280883128A01372024308700DC
:1016500006308500831629088312A3008316280804
:1016600083128A01372025308700063085008316D3
:1016700029088312A3008316280883128A013720C1
:101680002C30870006308500831629088312A300BA
:101690008316280883128A013720243087000730F8
:1016A0008500831629088312A30083162808831255
:1016B0008A01372087018501831629088312A30038
:1016C0008316280883128A013720243087000730C8
:1016D0008500831629088312A30083162808831225
:1016E0008A01372087018501831629088312A30008
:1016F0008316280883128A01372024308700073098
:101700008500831629088312A300831628088312F4
:101710008A01372087018501831629088312A300D7
:101720008316280883128A0137200130850083162A
:1017300029088312A3008316280883128A01372000
:101740000830870001308500831629088312A30022
:101750008316280883128A01372001308700013060
:101760008500831629088312A30083162808831294
:101770008A0137200330850001308700831629084D
:101780008312A3008316280883128A0137201130A0
:10179000870003308500831629088312A30083166F
:1017A000280883128A013720133087000330850010
:1017B000831629088312A3008316280883128A013E
:1017C00037201330870007308500831629088312DD
:1017D000A3008316280883128A013720333087003C
:1017E00007308500831629088312A3008316280872
:1017F00083128A013720373087000730850083162F
:1018000029088312A3008316280883128A0137202F
:1018100087018501831629088312A30083162808EF
:1018200083128A01372037308700073085008316FE
:1018300029088312A3008316280883128A013720FF
:1018400087018501831629088312A30083162808BF
:1018500083128A01372037308700073085008316CE
:1018600029088312A3008316280883128A013720CF
:1018700087018501831629088312A300831628088F
:1018800083128A0137200800023087000230850069
:101890006508A30064088A013720013087000430FE
:1018A00085006508A30064088A0137202830870076
:1018B00085016508A30064088A0137200430870089
:1018C000013085006508A30064088A0137200230D2
:1018D0008700023085006508A30064088A0137206C
:1018E00001308700043085006508A30064088A0180
:1018F00037202830870085016508A30064088A0125
:10190000372014308700013085006508A300640883
:101910008A01372008006430E600E701850187016D
:101920006708A30066088A0137200430870067082B
:10193000A30066088A013720063087006708A300E5
:1019400066088A013720073087006708A300660809
:101950008A0137200F3087006708A30066088A01D4
:1019600037200F308700013085006708A300660824
:101970008A0137200F308700033085006708A300F5
:1019800066088A0137200F30870007308500670816
:10199000A30066088A0137202F30870007308500B2
:1019A0006708A30066088A0137203F3087000730A8
:1019B00085006708A30066088A0137203B3087004E
:1019C000073085006708A30066088A0137201930B0
:1019D0008700073085006708A30066088A01372062
:1019E00008308700033085006708A30066088A0175
:1019F00037208701013085006708A30066088A0147
:101A0000372008008701013085006908A3006808B5
:101A10008A01372002308500083087006908A3005A
:101A200068088A0137200430850001308700690882
:101A3000A30068088A0137208501103087006908F3
:101A4000A30068088A013720043085000130870030
:101A50006908A30068088A013720850122308700C1
:101A60006908A30068088A013720043087006908E4
:101A7000A30068088A013720223087006908A30084
:101A800068088A0137200430850001308700690822
:101A9000A30068088A013720850110308700690893
:101AA000A30068088A0137200430850001308700D0
:101AB0006908A30068088A013720023085000830D1
:101AC00087006908A30068088A01372008000430ED
:101AD00087006B08A3006A088A013720203087003E
:101AE0006B08A3006A088A0137208701043085004B
:101AF0006B08A3006A088A013720023085006B0852
:101B0000A3006A088A0137208501103087006B081E
:101B1000A3006A088A013720023087006B08A300FF
:101B20006A088A013720013087006B08A3006A0821
:101B30008A013720083087006B08A3006A088A01F1
:101B400037208701013085006B08A3006A088A01ED
:101B50003720023085006B08A3006A088A0137200D
:101B6000043085006B08A3006A088A0137208501CC
:101B7000203087006B08A3006A088A0137201030E4
:101B800087006B08A3006A088A01372008308700A5
:101B90006B08A3006A088A013720013087006B08B0
:101BA000A3006A088A013720023087006B08A3006F
:101BB0006A088A013720043087006B08A3006A088E
:101BC0008A013720243087006B08A3006A088A0145
:101BD000372024308700043085006B08A3006A0892
:101BE0008A01372024308700063085006B08A30067
:101BF0006A088A01372006308500343087006B0878
:101C0000A3006A088A013720363087000630850035
:101C10006B08A3006A088A01372037308700063036
:101C200085006B08A3006A088A013720063085000A
:101C30003F3087006B08A3006A088A0137203F30D5
:101C40008700073085006B08A3006A088A013720E7
:101C5000063085003F3087006B08A3006A088A01C0
:101C600037203F308700043085006B08A3006A08E6
:101C70008A0137203F30870085016B08A3006A087E
:101C80008A0137201F3087006B08A3006A088A0189
:101C900037200F3087006B08A3006A088A013720BD
:101CA000073087006B08A3006A088A0137200630D6
:101CB00087006B08A3006A088A0137200430870078
:101CC000080002308700023085006D08A3006C0810
:101CD0008A01372004308700013085006D08A30099
:101CE0006C088A0137202830870085016D08A30021
:101CF0006C088A01372001308700043085006D08A8
:101D0000A3006C088A01372002308700023085006A
:101D10006D08A3006C088A01372004308700013069
:101D200085006D08A3006C088A01372028308700E1
:101D300085016D08A3006C088A01372011308700E7
:101D4000043085006D08A3006C088A013720080064
:101D50008501023087006F08A3006E088A013720D2
:101D6000013087006F08A3006E088A013720083011
:101D700087006F08A3006E088A01372087010130B1
:101D800085006F08A3006E088A01372002308500A5
:101D90006F08A3006E088A013720043085006F08A1
:101DA000A3006E088A0137202030870085016F0864
:101DB000A3006E088A013720043087006F08A30053
:101DC0006E088A013720123087006F08A3006E0862
:101DD0008A013720113087006F08A3006E088A013E
:101DE0003720183087006F08A3006E088A0137205B
:101DF00010308700013085006F08A3006E088A014B
:101E0000372010308700023085006F08A3006E086D
:101E10008A01372010308700043085006F08A30046
:101E20006E088A0137203030870085016F08A300D3
:101E30006E088A013720143087006F08A3006E08EF
:061E40008A0137200800B2
:02400E00FC3F75
:00000001FF
